:1000000099C0FFFF00C00FB617EE12BF739580FFB7
:100010000BC00894809B88944795783019F4112779
:1000200019BF82600FBE1895713011F49198FACF04
:100030007A3029F4919A112719BF8160F3CF40FDDE
:10004000919A40FF91984695EDCF81E012E013BF61
:10005000899A889808958827772712E019BF80FF2A
:10006000FECF0895809BFECF8099FECF13EE12BF86
:1000700012E018BF19BF772781FFFECF8D7F08954B
:100080002FEF2A95F1F71A95D9F70895332718E03D
:10009000F0E0331F10F4C69A01C0C698FF0FB5995F
:1000A000F160C79A26E02A95F1F7C79823E02A95D0
:1000B000F1F71A9571F73F2F089500001FED17BB58
:1000C000C798C49A1FEFDCDFC4981FEFD9DF3CEA62
:1000D000DEDF33E5DCDF0032B8F00023AAF0A0E277
:1000E000D5DF333599F030E0D2DFC79A26E02A9584
:1000F000F1F7C79823E02A95F1F73CEAC8DF33E52A
:10010000C6DFAA9569F702C030E0C1DF30E0BFDF8B
:1001100010E1B6DF089541E49EDF46E59CDF42E54D
:100120009ADF40E298DF49E496DF43E594DF40E55B
:1001300092DF089511271BBF1FEF12BBC49A18BB93
:1001400010E117BB82DF78948DDF4B31E9F3443542
:1001500019F488DF042F41C1433511F4DCDFF4CFFB
:10016000463529F442E377DF42E375DFEDCF4637CA
:1001700029F441E670DF40E66EDFE6CF443729F52B
:1001800045E569DF46E567DF43E165DF40E263DFC0
:1001900048E261DF48E35FDF48E45DDF4CE45BDFBA
:1001A00044E359DF40E357DF4CE655DF48E653DFD1
:1001B00045E651DF40E64FDF44E64DDF41E44BDFEB
:1001C00042E449DF40E047DFBFCF403719F443E561
:1001D00042DFBACF413619F449E53DDFB5CF4837A4
:1001E00009F4FBC0493709F4F8C0053509F10635B3
:1001F000F9F00331E9F00032D9F00832C9F00833E0
:10020000B9F00834A9F00C3499F0043389F00033C4
:1002100079F00C3669F0083659F0053649F00036A9
:1002200039F0043629F0023419F0013409F0D2C053
:10023000403511F442DFD1C0433471F413DF38E4A8
:1002400026DF362F24DF352F22DF342F20DF11E089
:100250002227510F621F0BC04336B1F403DF30E495
:1002600016DF362F14DF352F12DF342F10DF013465
:1002700051F0053641F0023431F0003621F00436F9
:1002800011F010E2FDDEA9C0423599F438E2FFDE3C
:10029000362FFDDE352FFBDEF9DE432FDCDE30E2CC
:1002A000F6DE362FF4DE352FF2DEF0DE432FD3DE1E
:1002B00024C0413429F4D6DE642FD4DE542F8DC0FF
:1002C000443481F4CFDE30ECE2DE362FE0DE352F31
:1002D000DEDE342FDCDE10E2D3DE11E02227510F08
:1002E000621F7BC0443671F430EAD1DE362FCFDE98
:1002F000352FCDDECBDE432FAEDE11E02227510FAE
:10030000621F22CF4C3421F410E117BBC49A65C0A0
:10031000453659F43CEABBDE30E8B9DE34E0B7DEFE
:1003200030E0B5DE10E3ACDE58C04C3671F49ADE36
:100330003CEAADDE342F3670306EA9DE30E0A7DE49
:1003400030E0A5DE10E39CDE48C0433789F4B2E01C
:1003500005D0B1E003D0B0E001D0F6CE30E397DEB7
:1003600030E095DE3B2F93DE91DE432F74DE08955F
:100370004D3659F43CE48BDE362F89DE352F87DE8F
:1003800030E085DE1FEF7CDE28C04A3359F46ADE98
:10039000C42F68DED42F66DEE42F442710D01FEF71
:1003A0006FDE1BC04E32B1F45DDEC42F5BDED42F96
:1003B00059DEE42F57DE03D01FEF62DE0EC03C2F64
:1003C00066DE3D2F64DE3E2F62DE342F60DE4F2F6F
:1003D00042DE08954FE33FDEB7CE4DE03CDEB4CEC3
:1003E0000000133029F0000000001A951330E9F7DF
:1003F0000895FFFFFFFFFFFFFFFFFFFFFFFFFFFF6E
:00000001FF
